:1000000075C099C098C097C096C096C094C093C060
:1000100092C091C090C08FC08EC08DC08CC00000B7
:1000200000000000000000000000000023456C9864
:10003000C9FF040714233764A0FFFFFFFFFFFFFF82
:10004000FFFFFFFFFF000000000000000000234052
:100050005F7AB4FFFFFFFFFFFF00140008140008E1
:100060000E140004080E14000305080E1400040802
:100070000A0E1114000305080A0E101400030508E7
:100080000A0E1012140008000E00080E0004080EDC
:10009000000305080E0004080E1100080E1100F3FD
:1000A000F404080E10121400080A0C0E0F1012149B
:1000B00000080EED14000203040500041400040EF1
:1000C0001400040810140004080F1114000305089C
:1000D0000A0E0004080A0E00EEEDECEB140E080404
:1000E0000004080E00EBECEDEEF3F41411241FBE37
:1000F000CFE5D2E0DEBFCDBF20E0A0E6B0E001C09A
:100100001D92A937B207E1F7EAE7F0E085E58087BD
:1001100081E0838314821282868311828BE081873F
:1001200088E58287E0E6F0E08DEF87838EEF8583B8
:10013000712CAAD0BFC164CF189525B7277E25BFE3
:1001400029B7226029BF21E022BF019728F020E1D2
:1001500088952150E9F7F9CF089588EE93E0EDCF27
:10016000369A3699FECF85B10895CF93C72D81E099
:10017000870D8F73782E662D90E08ED16FEF8C2FC8
:1001800090E0CF9189C1FF920F931F93CF93DF939C
:10019000F82E0BE710E0CEE7D0E0F11005C0CE015D
:1001A00073D1F801808304C0F8016081CE0174D15D
:1001B00021970F5F1F4FC437D10579F7DF91CF919A
:1001C0001F910F91FF900895D0DF81E0DCCF811166
:1001D00004C01BBC19BC18BC0895815090E0FC0100
:1001E000E25EFF4FE491EBBDFC01EE5CFF4FE4915A
:1001F000E9BDFC01EA5BFF4F849188BD08950F9330
:100200001F93CF93C82F8B01CC2369F085E0DFDFEC
:10021000C80193DF1BBC19BC18BCC8018EDFC80124
:100220008CDFC150F1CFCF911F910F910895CF93E3
:10023000DF93D82F64E170E08AE0E1DF84EF91E0A2
:100240007CDF8D2F64E614D1CAE06C2F11D1892F89
:1002500068EC70E0D4DF81DF8D2F6C2F09D1D92FAE
:1002600007D1892F68EC70E0CADF77DF68EC70E0B7
:100270008D2FC5DF72DF64E170E08AE0C0DF84EFBC
:1002800091E0DF91CF9159CF1092790083EA87B93D
:1002900086EC86B93699FECF369A3699FECF85B16F
:1002A0008095582E87E790E0EFD0853519F0612CC6
:1002B0008BDF11C0712C872D90E0E6D0682E8F3F28
:1002C00019F080E060DF07C0872D91E0970D792E4F
:1002D000803488F3F6CF90918300D0917D00109107
:1002E0007E00C0917B00CC2319F010E0D0E09AE1B1
:1002F0009F5F80E040E050E06AE570E0992379F08C
:100300009B012F5F3F4FF9013197E491EE2319F0E4
:10031000822F861BF6CF9150AB01B901EFCF982FFA
:100320006D2F70E0A82FB0E0E92FF0E0112321F04D
:100330009D012E1B3F0B05C09F0121503109260F47
:10034000371F3197E40FF51F049127593F4FF901EB
:100350000083915049F78D0F80938500DD2371F064
:10036000112329F0282F30E02150310902C020E06C
:1003700030E0F901E759FF4F91E0908397E0980F43
:10038000292F2150E22FE81BF0E0EB51FF4FE491C1
:10039000A22FB0E0A759BF4FEC932813F2CFE92F5B
:1003A000F0E0E859FF4F21E04091690030814313AC
:1003B00020E0921B90938600262D253FE8F5352DF1
:1003C0003134B0F4909187009F3F29F480917900F7
:1003D0008093870006C091E0960D692E981708F06B
:1003E000612C809187008F5F8F718093870024C07C
:1003F00020917900209387003F3AC0F4209180003B
:10040000222311F0CC2339F091E0960D692E981734
:1004100098F0612C11C0262D6816D9F3662019F0CA
:100420002150622E09C09150692E06C0C111F1CF32
:1004300080917C00882369F38FEF8DBD80E68CBDB1
:100440008FE384BB8BE187BB88EE88BB81E083BFF1
:1004500091EA9ABD80BF85B7806285BF789497B9CD
:1004600086EC86B98CE291E068DE7ADEE0DEFACFD7
:10047000991B79E004C0991F961708F0961B881FF6
:100480007A95C9F780950895E199FECF9FBB8EBB01
:10049000E09A99278DB30895262FE199FECF1CBAD3
:1004A0009FBB8EBB2DBB0FB6F894E29AE19A0FBEAC
:0804B00001960895F894FFCFB6
:00000001FF
